:10740000E0E0F0E0859194910196089520E82093C2
:1074100061001092610081E085BF82E085BF80EF4E
:1074200085B987EE84B91DB8769A10BA80EF81BB12
:1074300084E68BB985EF8AB980E58CBD81E08DBD8E
:10744000089580EE8BB98BEA57D0109289008AEFAD
:107450008093880082E080936F0083E080938100B6
:10746000E7E0F1E05ED0ED30E9F7A7E0B4E0EDE071
:10747000F1E003E010E101900D921A95E1F7A059B7
:10748000BF4F0A95B9F756D081E08093D7008AE4C0
:1074900082BF1092D8001092E2001092DA0010928F
:1074A000E10080E808D019BC1EBA1092E00070D448
:1074B00089E05CD481E98093D8000895F201F999BC
:1074C000FECFF2BDE1BD0895F9DFF89A80B508C09E
:1074D000F5DF1FBA80BD0FB6F894FA9AF99A0FBE7D
:1074E00031962F010895AFECB1E090E81BD08D9359
:1074F0009A95E1F7089586E008D010C083E005D0A2
:107500008F2F10D08E2F0ED080E05E9A5A980AC02E
:1075100005D085E0FADF06D080FDFDCF5A9A5E984F
:10752000089581918EBD8DB5000087FFFCCF8EB58B
:107530000895F4DFEFECF2E090EB5C98892FF2DF36
:1075400080E1F0DF5C9AEDDF8FEC8E278F77D9F743
:107550009395983B91F70895EDEBF1E0819190813F
:10756000019690838293092E0AF400940091BB0146
:1075700006FB5EF00096929111F493959083000CB7
:10758000081620F42E982F982D980895937009F4DA
:107590002E9A913009F42F9A923009F42D9A089579
:1075A000E4EBF1E097819923EAF08FB18095807F39
:1075B000669B88601C9B84609581891310C09681AE
:1075C000992381F49381891306C09481992396E9C4
:1075D00059F080E00AC083839095892304C0858395
:1075E0009AE0968380E09FEF948382830895809150
:1075F000BB0186FF2E9A2F9A2D9A22243324E4EB86
:10760000F1E0108611861286EFECF1E08091B60170
:1076100087FD36C084FD4DC082FF08952684222058
:10762000E1F3F894C089D78520E030E080E090E471
:10763000AFEFBFEF119682199040E0F72D0100E007
:107640001FE627FD13C0ECE6F4E011928EE781936C
:1076500092E491939AE5E11708F092E4E03BC9F7D0
:107660008193108266DFFE01219648DF3CDFF9013D
:1076700021D320583F4F040D151D2A9411F7ABC19B
:107680008301282D6090D8017090D70146D019F45D
:107690008823C1F70895380188243FD0E1F580910F
:1076A000D601821709F483016090DA017090D90144
:1076B000F4CF6090DA017090D9012FD081F4882343
:1076C000C1F708959FEF85FD08C086FD05C083FFC3
:1076D000089596DEE9F37FC191E097FB890E662459
:1076E00077248301222719D0B1F4882389F380916C
:1076F000D60136F0881650F4821730F0213003C0DE
:10770000881520F4281710F48301282F6090DA01DF
:107710007090D901E8CF3801822EF301EFDEE3DE6D
:10772000CFECD1E0E0E0F1E097E00990819108161C
:1077300021F49A95D1F708808010F0CEC9E0D5DE0B
:0A774000CA95E9F7F6DE88270895E0
:10774A0041524455424F59C82F258113AF0000FFBB
:10775A00FFCFCFFFFFFFFFCFCFFFFF0000FE067E68
:10776A007E06FE46565616FE0656461EFE3F61E940
:10777A00E3FFE3EBE3FFE3EBE3FFE16B3F1201100F
:10778A00010200000841233700010000010001093D
:10779A00023E0002010080320904000001020201D7
:1077AA000005240010010424020405240600010730
:1077BA000582030800FF09040100020A000000070D
:1077CA0005040210000107058302100001040309E1
:1077DA00042203410072006400750069006E006FA4
:1077EA000020004D006900630072006F0020002035
:0477FA00002000006B
:1078000011241FBE8DEF9AE09EBF8DBF04B714BE3A
:1078100088E18093600010926000409100085091D0
:1078200001086F917F91A6C00F928F939F931F9233
:107830000FB60F9211244F936F938091DA0080FF5F
:107840004CC038C00F920FB68F939F93EF93FF9366
:1078500088278093850080938400E4EBF1E0978192
:10786000907261F490818917980B908309F45D9868
:1078700091818917980B918309F4289896819150EA
:1078800008F096839481915008F09483881639F417
:107890007C9B05C0B5DD19F0C10101961C01FF916B
:1078A000EF915CC080E189BD82E189BD09B400FE31
:1078B000FDCF08958091D80080FF0FC08091DA003D
:1078C0008E7F8093DA008091D90080FF04C0EADFC8
:1078D00081E08EBB02C019BC1EBA8091E10080FF1E
:1078E0000BC03ED280FF08C03ED28091D80080629B
:1078F000E2DD19BC85E08EBB8091E10084FF1AC0F7
:107900002FD284FF17C0CEDF8091D8008F7DD3DDCA
:107910008FEE2AD025D28F7E816028D28091BF0140
:10792000882331F48091E30087FD02C081E001C02B
:1079300084E08EBB8091E10083FF0CC011D283FFF5
:1079400009C087EF11D082E08EBB1092BF010BD02F
:107950000AD21ED26F914F910F901F909F918F91DD
:107960000FBE0F9018958EEF0090E1000822009254
:10797000E10008954BDDA0E0B1E0EAE4F7E705900F
:107980000D92A33BE1F71D92BB30E9F701FD0FC05B
:1079900000FF03C07C9B0BC008C003FF08C06757F3
:1079A000774729F04757574711F02ADDA1F449DD01
:1079B0002224332431018824B0DE789447D007D3C1
:1079C000EFDD80DE811411F012DEF8CFC5DDC101DC
:1079D000805B964398F3F89489EB8EDD81E0809389
:1079E000E00010926F0010928100109285001092BA
:1079F000840081E085BF15BEC5DD5D9828980C9494
:107A00000000A9D107C054D102C0DED239F0A5D1FF
:107A100082FFFBCF85FFF7CF8091F1000895082EFC
:107A200083E09AD185FD07C08FD102C0CDD269F025
:107A300094D180FFFBCF0092F1008091BB0185FBC8
:107A400026F05D9A84E68093B401089584D182FF84
:107A50004CC18091BB0185FB26F0289A84E6809377
:107A6000B501CFDF182F853431F48CEB94E31C0182
:107A700025DD8DE008C1843511F4C3DFFACF8C34E5
:107A8000C1F38035B1F3843721F484E4C8DF80E0AA
:107A9000FAC0813611F489E5F6C0813429F4B1DFEA
:107AA000582EAFDF482EE5CF803711F483E5EBC0C9
:107AB000833539F4C0E0D1E08991B1DFC730E1F717
:107AC000E3C0863521F481E3AADF84E3DCC0863796
:107AD00061F481E3669B8E5F1C9B8F5FA0DF8FB19B
:107AE000809582958F708F5BCEC08837A9F489DF2F
:107AF0008093BB01289884FD289A5D9883FD5D9A48
:107B00002E9881FD2E9A2F9882FD2F9A2D9880FD18
:107B10002D9A87FD8824ADCF8A3649F48FE9F5DCAC
:107B2000C3E000DD7CDFCA95E1F7F8DCADC0833748
:107B300031F487E874DF85E972DF8EE1A4C0853611
:107B400039F4E0E8F3E7C9D0E058F040E0F791CF2E
:107B5000823631F489E563DF80E061DF80E893C03D
:107B6000823419F0873609F07AC02224332449DFA1
:107B7000D82F47DFC82F45DF082F8354843008F003
:107B800081C0063411F4440C551CF20110926F00B0
:107B90001736A1F4033471F483E0B1DCC3DC3FDFBA
:107BA0002197E1F7BBDC08C0063411F4859101C0D0
:107BB0008BDC35DF2197C2F72F0149C00334A1F4D4
:107BC0008E2F8F7021F497DC80E299DCA1DC93DCAE
:107BD00082E095DC16DFA6DCCA95E1F799DC3196E8
:107BE000DA9571F72F0131C00634F1F49F01F437B3
:107BF000D8F473D019C005DF063461F4C0FB46F039
:107C0000F43728F4182E81E087BFE89511243296C6
:107C1000082E0AC0043439F4DF01B370A153BD4FFC
:107C20008D93319601C054DC21972AF7043431F446
:107C30002F01F370FE2B49F47DDC07C0063429F4D4
:107C40002F01F901F43708F446D08DE0E8DE063460
:107C500011F45694479482E080936F0015C08237E8
:107C6000E1E049F08634E0E031F08E34E3E019F0F1
:107C7000813531F4E2E0F0E089E087BF849103C010
:107C80008B3111F08FE3CBDE83E0AED15DD095FF79
:107C900003C009C099D149F160D080FFFBCF54D017
:107CA00002C092D111F159D080FFFBCF84E09CD16A
:107CB0008BE74BC0AFECB1E0F437B8F40ED090E4F2
:107CC0000D901D9081E087BFE89532969A95C1F797
:107CD0001124E058F04085E001C083E001D081E14B
:107CE00087BFE89507B600FCFDCF08959091C701C6
:107CF0008091C801913231F0913A61F5813251F5AC
:107D000038D082C0803231F534D05ED1E9F0853090
:107D1000D9F023D083FD18C082FFF7CF04C07CDEEA
:107D20008193615031F09091F3008091F200892BA2
:107D3000B1F7BEDF611549F704C046D129F085309F
:107D400019F00BD080FFF9CF8EE79091E8008923DE
:107D50008093E800089584E047D18091E800089579
:107D60008091E2000895FCDF8E7F80618093E200C5
:107D7000089528D1E0ECF1E067E0089582E061EC3D
:107D800009D083E061E802D084E060E842E103C00A
:107D900080E060E042E028D181E007D01092ED0061
:107DA0006093EC004093ED0008959091EB00892BD7
:107DB0008093EB00089560E0923039F0933041F009
:107DC000913071F4EDE362E10BC0EFE46EE308C0C3
:107DD000813018F4EDE864E003C011F4E1E962E2F7
:107DE000F1E008958091C70188234CF402C0ECD0E3
:107DF00051F0B3DF82FFFBCF5BCFE6D021F0ADDFE8
:107E000080FFFBCFA1DF08954091CD015091CE01BD
:107E10004617510510F490E028C0611511F0462F67
:107E2000FACF92DF40E0F7CFCFD059F1853049F15A
:107E300094DF83FD3DCF91DF82FD20C080FF15C020
:107E40003091F3002091F20005C081918093F10000
:107E500041502F5F411519F028303105B0F350E043
:107E60002830310509F451E06FDF4115E9F655235B
:107E7000D9F604C0A9D029F0853019F06EDF82FF51
:107E8000F9CF16CFE7ECF1E0C7DD8193EF3CE1F7E6
:107E90002DDF63DF83FF91C08091C7019091C801FE
:107EA000913009F170F09330F1F0953009F444C04D
:107EB000963009F456C0983009F460C0993059F7EB
:107EC00067C0823841F78091CB018DD02091EB00C3
:107ED0001092E90077D02295269521702093F10029
:107EE0001092F10052C0882311F08230A1F68F71F8
:107EF000823089F68091C9018823D1F42091CB0189
:107F0000277049F22093E9008091EB0080FF10C0B8
:107F1000933011F480E20BC080E147DF81E0880FED
:107F20002A95E9F78093EA001092EA0088E03DDFA5
:107F30001092E90047D02AC0882391F41091C9011A
:107F400010680FB7F8943ED04DDF07DF80FFFDCFFC
:107F50001093E300103883E009F482E08EBB0FBF7A
:107F60002CC08058823048F58091C9019091CA0197
:107F700022DF603011F126D047DF1FC08038E9F4DE
:107F800021D08091BF018093F100DEDE2BDF15C090
:107F9000882399F49091C901923078F49093BF01AD
:107FA00011D020DF8091BF01882321F48091E3006C
:107FB00091E087FD94E09EBBE1DECFDE83FF089574
:107FC00080E2F3DE87EFC1CE8EB388230895FCDF15
:107FD00069F08091E9008F931092E900BEDE83FF83
:0E7FE00001C050DF8F9187708093E9000895F3
:047FFC005DCEFBDC7F
:040000030000740085
:00000001FF
